:020000040800F2
:10000000709000209D010008310D00089D0A000835
:100010002D0D0008950300081112000800000000D3
:10002000000000000000000000000000AD0E00080D
:100030004D05000800000000410D0008B501000852
:10004000B7010008B7010008B7010008B7010008B0
:10005000B7010008B7010008B7010008B7010008A0
:10006000B7010008B7010008B7010008B701000890
:10007000B7010008B7010008B7010008B701000880
:10008000B7010008B7010008B7010008B701000870
:10009000B7010008B7010008B7010008B701000860
:1000A000B7010008B7010008B7010008B701000850
:1000B000B7010008B7010008B7010008B701000840
:1000C000B7010008B7010008B7010008B701000830
:1000D000B7010008B7010008B7010008B701000820
:1000E000B7010008B7010008B7010008B701000810
:1000F000B7010008B7010008B7010008B701000800
:10010000B7010008B7010008B7010008B7010008EF
:10011000B7010008B7010008B7010008B7010008DF
:10012000B7010008B7010008B7010008B7010008CF
:10013000B7010008B7010008B7010008B7010008BF
:10014000B7010008B7010008B7010008B7010008AF
:10015000B7010008B7010008B7010008B70100089F
:10016000B7010008B7010008B7010008B70100088F
:10017000B7010008B7010008B7010008B70100087F
:10018000B7010008B7010008DFF80CD000F064F8F0
:1001900000480047B51E00087090002006488047C0
:1001A00006480047FEE7FEE7FEE7FEE7FEE7FEE75C
:1001B000FEE7FEE7FEE7FEE70911000889010008F7
:1001C000421C10F8011B0029FBD1801A704770B542
:1001D000064601F07BFC046805460A2200213046F1
:1001E00000F002F82C6070BD2DE9F04791460F46F3
:1001F00080460446002614F8015B2DB100F03EF85D
:100200000068405DC007F6D12B2D02D02D2D18D0EF
:10021000641E4A463946204600F034F827B1396852
:10022000A14201D1C7F8008071054FF002040BD53F
:100230004042002803DD01F049FC0460A007BDE84E
:10024000F08746F48066E4E70028F8DA01F03EFC27
:1002500004606FF00040F2E7064C074D06E0E068EE
:1002600040F0010394E8070098471034AC42F6D3FD
:10027000FFF78EFFFC6300081C640008004870470D
:100280005C6300082DE9F05F824600780027154680
:100290008B460AF10104B946302801D09DB113E024
:1002A00014F8010B0127782803D0582801D045B154
:1002B0000AE00DB1102D07D10027102514F8010B0D
:1002C00002E0082500E00A250026B0460EE005FB06
:1002D000080005FB06F1012701EB10461FFA80F824
:1002E000B6F5803F00D3B94614F8010B294600F05B
:1002F00018F80028EBDABBF1000F05D00FB1641E2F
:1003000000E05446CBF80040B9F1000F06D001F0F0
:10031000DDFB02210160C81EBDE8F09F48EA0640EF
:10032000FAE73A2800D2303820F02002412A01D3DF
:10033000A2F13700884201D34FF0FF30704770B50B
:100340008C1810F8015B15F0070301D110F8013B80
:100350002A1106D110F8012B03E010F8016B01F807
:10036000016B5B1EF9D12B0705D40023521E0DD45F
:1003700001F8013BFAE710F8013BCB1A921C03E0AD
:1003800013F8015B01F8015B521EF9D5A142D8D3E5
:10039000002070BD00BFFEE70146302905DB39298A
:1003A00003DCA1F13000C0B27047612905DB66298A
:1003B00003DCA1F15700C0B2F6E7412905DB46296D
:1003C00003DCA1F13700C0B2EEE73720ECE7000014
:1003D00010B5394800683949884208D23648001DAE
:1003E00037490860001F00683649086001E000F0E6
:1003F000F9FD35A000F05CFD002858D035480068B4
:1004000000785B2804D133480068401C31490860FB
:10041000002404E000F0D6FA2F490855641C042C8F
:10042000F8DB2EA000F044FDA8B12A48006800784F
:100430005B2804D127480068401C26490860002436
:1004400006E000F0BFFAC1B2234808300155641C31
:10045000042CF6DB08E0FF201F490872FF211E482C
:10046000417200218172C1721FA000F021FDA8B16C
:100470001848006800785B2804D116480068401CC2
:1004800014490860002406E000F09CFAC1B212484A
:10049000001D0155641C042CF6DB0BE000200E4906
:1004A000087100210C4841718171C17102E000F0B6
:1004B00099FD10BD00BFFCE700000E08C0D401008C
:1004C000D0000020C4000020435F49505F414444F5
:1004D00052000000EC000020E4020020435F49507D
:1004E0005F4D41534B000000435F49505F4741540B
:1004F0004500000010B500220268134B1A40CC687A
:100500000B6823434C6923438C692343CC69234301
:100510000C6A23434C6A23438C6A23434C6B23436A
:100520008C6B23431A430260426922F00702D1E92F
:100530000B3423431A4342610B6943604B68836069
:100540008B68C36010BD00003F801CF07047000046
:1005500001490860704700000C3C024070B5044639
:100560000A460026082502B909E0012A01D116022F
:1005700005E0022A01D1160201E04FF4407600F0B6
:1005800097F80546082D28D11548006820F44070DA
:100590001349086008460068304308600846006850
:1005A00020F0F80008600846006844F002010843A3
:1005B0000B4908600846006840F48030086000F08D
:1005C00077F805460648006820F0020004490860F4
:1005D0000846006820F0F8000860284670BD00005A
:1005E000103C024008201049096801F48031B1F53F
:1005F000803F01D1012015E00B49096801F010018D
:1006000009B105200EE00849096801F0EF0109B1C0
:10061000062007E00449096801F0020109B107203A
:1006200000E00820704700000C3C024003480068CE
:1006300040F000400149086070470000103C024053
:1006400030B502460C46082500F032F80546082D64
:1006500017D10D48006820F440700B490860084627
:10066000006808600846006840F0010008601470E7
:1006700000F01EF805460448006820F00100024919
:100680000860284630BD0000103C02400548006864
:1006900000F0004028B1044802490C3908600348C2
:1006A00008607047103C024023016745AB89EFCDDD
:1006B00008B508200090FFF795FF009002E0FFF7D3
:1006C00091FF00909DF800000128F8D09DF80000EF
:1006D00008BD000010B50446FFF7D8FFF320FFF770
:1006E00037FF02211820FFF739FF00201B4908605F
:1006F00025E01A480068205C7D2800D123E01748D7
:100700000068205C202800D11DE014480068205CAF
:100710000A2800D117E011480068205C0D2800D19C
:1007200011E00E4A1268A15C0C4A12680C4BD018FA
:10073000FFF786FF09480068401C08490860074821
:100740000068FF28D5D900BF04490968044A881801
:100750000021FFF775FFFFF769FF10BD9000002033
:1007600000C0000810B50446FFF790FFF320FFF724
:10077000EFFE00204549086080E045480068454993
:10078000884207D102212020FFF7E8FE082801D087
:1007900000BFFEE73E4800683F49884207D102217A
:1007A0002820FFF7DBFE082801D000BFFEE738480D
:1007B00000683A49884207D102213020FFF7CEFE77
:1007C000082801D000BFFEE731480068344988425C
:1007D00007D102213820FFF7C1FE082801D000BF51
:1007E000FEE72B4800682F49884207D102214020AC
:1007F000FFF7B4FE082801D000BFFEE724480068D8
:100800002949884207D102214820FFF7A7FE08287E
:1008100001D000BFFEE71E4800682449884207D186
:1008200002215020FFF79AFE082801D000BFFEE702
:10083000174800681749884216D3154800681C49B4
:10084000884211D21B4811490968405CFF280BD02F
:1008500018480E4A1268815C0D480068FFF7F0FEE8
:10086000082801D000BFFEE709480068401C08497D
:10087000086006480068401C044908600348006896
:10088000A042FFF47AAFFFF7D1FE10BD9000002028
:10089000E800002000000108000002080000040831
:1008A000000006080000080800000A0800000C0804
:1008B00000000E0843830020F0B50A460021002303
:1008C000002400BF3DE0012505FA01F3156805EAA3
:1008D00003049C4234D105684F000326BE40B54353
:1008E000056015794E00B5400668354305601579F9
:1008F000012D02D01579022D16D185684F000326EF
:10090000BE40B543856055794E00B5408668354395
:100910008560456801268E40B543456045689679F7
:100920008E40B6B235434560C5684F000326BE40D1
:10093000B543C560D5794E00B540C6683543C5603E
:10094000491C1029BFD3F0BDF0B5002300244D078A
:10095000ED0E02FA05F3CE1000F1200555F82650F1
:100960004E07F70E0F26BE40B543CF1000F120060C
:1009700046F82750CE1000F1200555F8265045EADC
:100980000304CE1000F1200545F82640F0BD418358
:1009900070470183704730B5024612F8010BFFF72C
:1009A000FBFC0446102C01DD002030BD1078FFF761
:1009B000F3FC0346102B01DD0020F6E703EB0410E7
:1009C000C0B2F2E710B50C48006800785D2801D18C
:1009D000002010BD08480068FFF7F9FB84B200BF93
:1009E00005480068017804480068401C024A10600D
:1009F0002C29F5D12046ECE7EC00002070B502254B
:100A00002248234908600846006800783A281BD12C
:100A100015E01F480068007853280BD11C48006877
:100A2000401C1B49086008460068FFF7D0FB0546DC
:100A3000284670BD16480068401C154908601448D7
:100A4000006800780028E4D11248114908600024A9
:100A500016E00F480068006800B90BE00C48006819
:100A600000680D49884200D90CE009480068056813
:100A70002846DEE7641C06480068001D044908603B
:100A8000082CE6D300BF2846D3E7000000C00008CA
:100A9000900000200078FF1F9999990000BFFEE7A1
:100AA00001464FF48042224B1A800A0A214B1A73E6
:100AB00000BF204A127A02F00102002AF9D01D4A32
:100AC000127B1C4B197300BF1A4A127A02F0010202
:100AD000002AF9D0174A127B0022164B1A7300BF66
:100AE000144A127A02F00102002AF9D0114A127B4C
:100AF0000122104B1A7300BF0E4A127A02F0010253
:100B0000002AF9D00B4A127B00220A4B1A7300BF4D
:100B1000084A127A02F00102002AF9D0054A107B35
:100B200000BF4FF48042024B9B1E1A8070470000AA
:100B30001A0C02400030014010B501464FF48040CD
:100B4000284B1880080A284B187300BF2648007AE3
:100B500000F001000028F9D02348007B224B1973D4
:100B600000BF2148007A00F001000028F9D01E489B
:100B7000007B00201C4B187300BF1B48007A00F05C
:100B800001000028F9D01848007B0220164B18738A
:100B900000BF1548007A00F001000028F9D0124883
:100BA000007B0020104B187300BF0F48007A00F044
:100BB00001000028F9D00C4B187B020200201873AA
:100BC00000BF0948007A00F001000028F9D0064B68
:100BD000187B02434FF48043024CA41E238010462E
:100BE00010BD00001A0C02400030014002464FF4D4
:100BF0008040214B1880100A204B187300BF1F48FB
:100C0000007A00F001000028F9D01C48007B1B4B43
:100C10001A7300BF1948007A00F001000028F9D0CB
:100C20001648007B8020154B187300BF1348007ACC
:100C300000F001000028F9D01048007B01200F4B84
:100C4000187300BF0D48007A00F001000028F9D0A9
:100C50000A48007B0948017300BF0848007A00F089
:100C600001000028F9D00548007B4FF48040024B7A
:100C70009B1E1880012070471A0C02400030014072
:100C800002464FF48040274B1880100A264B1873F9
:100C900000BF2548007A00F001000028F9D0224862
:100CA000007B214B1A7300BF1F48007A00F001003F
:100CB0000028F9D01C48007B80201B4B187300BF14
:100CC0001948007A00F001000028F9D01648007B8E
:100CD0000220154B187300BF1348007A00F0010082
:100CE0000028F9D01048007B080A0F4B187300BF8A
:100CF0000D48007A00F001000028F9D00A48007B76
:100D0000094B197300BF0848007A00F00100002861
:100D1000F9D00548007B4FF48040024B9B1E1880A1
:100D2000012070471A0C02400030014000BFFEE76E
:100D300070470000014908627047000000000E4241
:100D40007047000029B1064A12680243044B1A603A
:100D500004E0034A12688243014B1A6070470000A6
:100D60003038024029B1064A12680243044B1A6027
:100D700004E0034A12688243014B1A607047000086
:100D80004038024029B1064A12680243044B1A60F7
:100D900004E0034A12688243014B1A607047000066
:100DA0002038024029B1064A12680243044B1A60F7
:100DB00004E0034A12688243014B1A607047000046
:100DC0004438024029B1064A12680243044B1A60B3
:100DD00004E0034A12688243014B1A607047000026
:100DE0002438024021B1028842F04002028004E02F
:100DF00002884FF6BF731A400280704710B5044650
:100E00001148844208D101218014FFF7DBFF002143
:100E1000A014FFF7D7FF16E00C48844208D1012147
:100E20000014FFF7AFFF00212014FFF7ABFF0AE02B
:100E30000748844207D10121C013FFF7A3FF002117
:100E4000E013FFF79FFF10BD003001400038004065
:100E5000003C00400246002013890B400BB10120EA
:100E600000E0002070470146888970478181704703
:100E700010B50022028802F441520B884C882343AB
:100E80008C882343CC8823430C8923434C892343F8
:100E90008C892343CC8923431A430280838B4FF2EE
:100EA000FF74234083830B8A038210BD70470000C8
:100EB00002462A4800682A4B18604AE02848006821
:100EC000007800B946E0264800680078FF2800D185
:100ED00040E02348006800787D2800D13AE02048AF
:100EE00000680078222805D01D480068401C1C4B73
:100EF00018602EE01A480068401C194B186018460C
:100F000000680078137898421DD1002108E0505CF9
:100F1000134B1B685B5C984200D004E0481CC1B2D4
:100F2000505C0028F3D100BF505C60B90C480068E9
:100F3000405C222807D10A480368C81C1844084BA3
:100F400018600120704706480068401C044B186078
:100F500000BFB3E700BF0020F4E70000D00000208E
:100F6000EC00002010B503461D48036033E01C4828
:100F70000068007800B92FE0194800680078FF2861
:100F800000D129E01648006800787D2800D123E0D0
:100F90001348006800780C78A04217D100220DE0B9
:100FA000885C0F4C24682478A04200D009E00C48EB
:100FB0000068401C0A4C2060501CC2B2885C0028AB
:100FC000EED100BF885C08B9012010BD044800685C
:100FD000401C034C2060CAE700BF0020F5E700007A
:100FE000EC000020C0200C490870A82048700120A7
:100FF00088700220C870FF200872FF2106484172E5
:1010000000218172C1720020034908710021024849
:1010100041718171C1717047E40200200CB500205C
:10102000019000903448006840F4803032490860F4
:1010300000BF3148006800F4003000900198401C67
:101040000190009818B90198B0F5A04FF1D12A4845
:10105000006800F4003010B10120009001E0002091
:1010600000900098012846D123484030006840F0A5
:1010700080502149403108602048006840F44040D9
:101080001E4908601C48083000681B490831086088
:101090000846006840F4204008600846006840F4B4
:1010A000A05008601648091F0860081F006840F03B
:1010B0008070091F086000BF0F48006800F00070D2
:1010C0000028F9D040F205600E4908600A4808304F
:1010D000006820F0030008490831086008460068ED
:1010E00040F00200086000BF03480830006800F0CC
:1010F0000C000828F8D10CBD0038024000700040F8
:1011000019544007003C024010B51648006840F0F2
:101110000100144908600020124908310860114894
:101120000068114908400F4908601048091D08600F
:10113000081F006820F48020091F0860002009496A
:101140000C310860FFF76AFF4FF000600849086043
:1011500007488030006840F470000549803108601D
:1011600010BD000000380240FFFFF6FE10300024E2
:1011700008ED00E021B1028842F00102028004E0A3
:1011800002884FF6FE731A400280704700220288E0
:10119000184B98420ED0184B98420BD0B0F1804FAC
:1011A00008D0164B984205D0154B984202D0154BEB
:1011B000984204D14FF68F731A404B881A43124B52
:1011C000984207D0114B984204D04FF6FF431A4083
:1011D0000B891A4302804B68C3620B880385054B59
:1011E000984202D0044B984201D18B7A03860123A6
:1011F0008382704700000140000401400004004069
:1012000000080040000C00400010004000140040A6
:1012100000BFFEE730B503461D4801681D48008841
:101220001D4C246860830020087100BF087800F01E
:1012300001000028FAD008790B7100BF087800F08F
:1012400001000028FAD008790020087100BF087852
:1012500000F001000028FAD008790020087100BFD2
:10126000087800F001000028FAD008790202002076
:10127000087100BF087800F001000028FAD0087952
:101280000243044C2488044D2D682C83104630BD45
:10129000B4010020B8010020B001002030B50246A2
:1012A0000B461A4C2168012404EB8204E200184C1E
:1012B0002488184D2D686C8300240C7100BF0C78B5
:1012C00004F00104002CFAD00C790B7100BF0C78EB
:1012D00004F00104002CFAD00C790A7100BF0C78DC
:1012E00004F00104002CFAD00C7900240C7100BF2A
:1012F0000C7804F00104002CFAD0087900BF044CEB
:101300002488044D2D682C8330BD0000B4010020DA
:10131000B8010020B001002070B502460C461F48FD
:101320000168012000EB8200C2001D4800881D4DAD
:101330002D6868830020087100BF087800F0010064
:101340000028FAD008790C7100BF087800F001007D
:101350000028FAD008790A7100BF087800F001006F
:101360000028FAD008790020087100BF087800F042
:1013700001000028FAD0087903020020087100BF9C
:10138000087800F001000028FAD008790343044DE2
:101390002D88044E36683583184670BDB401002090
:1013A000B8010020B001002030B502460B461748B6
:1013B000016817480088174C246860830020087172
:1013C00000BF087800F001000028FAD008790A71FF
:1013D00000BF087800F001000028FAD00879042046
:1013E000087100BF087800F001000028FAD00879E1
:1013F0000B7100BF087800F001000028FAD00879CE
:10140000034C2488034D2D682C8330BDB40100208B
:10141000B8010020B001002030B503460A461C4840
:1014200001681C4800881C4C2468608300200871F7
:1014300000BF087800F001000028FAD008790B718D
:1014400000BF087800F001000028FAD008790420D5
:10145000087100BF087800F001000028FAD0087970
:10146000100A087100BF087800F001000028FAD0C7
:1014700008790A7100BF087800F001000028FAD04E
:101480000879044C2488044D2D682C8330BD00005D
:10149000B4010020B8010020B001002070B503465F
:1014A0000C4619480168012000EB8300C30017486F
:1014B0000088174D2D6868830020087100BF0878E8
:1014C00000F001000028FAD008790C7100BF0878FC
:1014D00000F001000028FAD00879181D087100BF3B
:1014E000087800F001000028FAD008790A7100BFDE
:1014F000087800F001000028FAD00879034D2D8803
:10150000034E3668358370BDB4010020B801002059
:10151000B001002070B503460C461E48016801204A
:1015200000EB8300C3001C4800881C4D2D686883B5
:101530000020087100BF087800F001000028FAD0F0
:1015400008790C7100BF087800F001000028FAD07B
:101550000879181D087100BF087800F00100002804
:10156000FAD00879100A087100BF087800F001006D
:101570000028FAD008790A7100BF087800F001004D
:101580000028FAD00879044D2D88044E366835833A
:1015900070BD0000B4010020B8010020B00100209F
:1015A0000549064A11604FF48041054A116005491A
:1015B000054A116070470000000C0240B001002095
:1015C000B801002008300140B401002010B5052208
:1015D00003216248FFF7B8F9052204215F48FFF7AD
:1015E000B3F9052211465D48FFF7AEF902205C49C8
:1015F0000871002088710220C871487108200860B5
:101600005648FFF759F92020554908605348FFF71D
:1016100053F91020524908605048FFF74DF95148DE
:10162000FFF7ECFB0020504908808880C8800881C3
:101630004FF40070488100208881C881072008820B
:101640004FF4827048804748FFF712FC012145485B
:10165000FFF7C8FB04204249086001200871002000
:101660008871022048714148FFF726F904213F485C
:10167000FFF78DF94FF440403949086001200871A7
:1016800000208871022048713948FFF715F94FF49E
:1016900040413748FFF77DF9012031490860087162
:1016A00000208871022048713048FFF705F90121B8
:1016B0002E48FFF76CF9002029490871C8714FF4D2
:1016C000006008602B48FFF7F7F84FF0C0602A4928
:1016D000086024480C304860284888600020C860B2
:1016E00093200861002048614FF4806088610020E9
:1016F000C861086248624FF4003088620020C86206
:10170000012008630020486388631D48FEF7F2FE4D
:101710004FF0C0601849086012480C304860194802
:1017200088604020C86093200861002048614FF421
:10173000806088610020C861086248624FF4003010
:1017400088620020C8620120086300204863886323
:101750000B481830FEF7CEFE10BD0000000402401A
:1017600064000020003001406802002000180240A0
:10177000000C0240001402407C020020438B002039
:10178000406402400001002010B5052203215A48A0
:10179000FFF7DAF8052204215748FFF7D5F80522AC
:1017A00011465548FFF7D0F802205449087100202F
:1017B00088710220C8714871082008604E48FFF700
:1017C0007BF820204D4908604B48FFF775F8102042
:1017D0004A4908604848FFF76FF84948FFF70EFB91
:1017E0000020484908808880C88008814FF4007034
:1017F000488100208881C881072008824FF48270C8
:1018000048803F48FFF734FB01213D48FFF7EAFAE3
:101810004FF4404039490860012008710020887168
:10182000022048713848FFF747F84FF440413648E6
:10183000FFF7AFF801203149086008710020887176
:10184000022048713148FFF737F801212F48FFF790
:101850009EF8002029490871C8714FF400600860A3
:101860002B48FFF729F84FF0C0602A490860244848
:101870000C304860284888600020C86079200861E2
:10188000002048614FF4806088610020C8610862D0
:1018900048624FF4003088620020C862012008636B
:1018A0000020486388631D48FEF724FE4FF0C060A7
:1018B0001849086012480C30486019488860402078
:1018C000C86079200861002048614FF48060886119
:1018D0000020C861086248624FF40030886200202E
:1018E000C862012008630020486388630B481830F1
:1018F000FEF700FE10BD000000040240640000205E
:101900000030014068020020000C02400018024034
:10191000001402407C020020438B002040640240FF
:10192000BC01002000B50920FFF706F900BD00B595
:101930000920FFF76FFC00BD10B504464FF480414D
:1019400001EB0421491C8AB202211046FFF74EF92F
:1019500000BF4FF4804202EB0422521C91B20846B1
:10196000FFF79EF80028F4D110BD10B504460222FE
:1019700001212046FFF792FD00BF01212046FFF71D
:101980008DFC0028F9D110BDF0B504460F46154670
:101990001E464FF4804101EB04218AB239461046BD
:1019A000FFF724F94FF4804101EB0421091D8AB2AD
:1019B00029461046FFF764F94FF4804101EB0421FA
:1019C00010318AB231461046FFF75AF94FF4804180
:1019D00001EB0421491C8AB201211046FFF706F9E8
:1019E00000BF4FF4804202EB0422521C91B2084621
:1019F000FFF756F80028F4D1F0BDF0B506460C46C6
:101A000017461D46224600213046FFF747FD3A465D
:101A100004213046FFF77EFD2A4610213046FFF7AD
:101A200079FD012211463046FFF738FD00BF012144
:101A30003046FFF733FC0028F9D1F0BD10B504465D
:101A400021780920FFF7D2F861780A20FFF7CEF855
:101A5000A1780B20FFF7CAF8E1780C20FFF7C6F851
:101A600021790D20FFF7C2F861790E20FFF7BEF84B
:101A700010BD10B5044621780920FFF795FC617868
:101A80000A20FFF791FCA1780B20FFF78DFCE1788D
:101A90000C20FFF789FC21790D20FFF785FC617987
:101AA0000E20FFF781FC10BD0FB4084610B5064AA2
:101AB00002A900F01EF8044602A9002000F02AF84E
:101AC000204610BC5DF814FB151B00080048704749
:101AD0003C02002002E008C8121F08C1002AFAD107
:101AE00070477047002001E001C1121F002AFBD19E
:101AF00070472DE9F04116460F460446002503E0E5
:101B00003946B047641C6D1C20780028F8D128465F
:101B1000BDE8F0810A68531C0B601070704710B567
:101B200004464FF4804101EB0421491C8AB2102184
:101B30001046FFF75BF800BF4FF4804202EB04222F
:101B4000521C91B20846FEF7ABFF0028F4D14FF4C7
:101B5000804101EB0421891C8AB2FF211046FFF766
:101B600045F810BD10B50446102201212046FFF7AC
:101B700095FC00BF01212046FFF790FB0028F9D11A
:101B8000FF2202212046FFF789FC10BD10B5044654
:101B90004FF4804101EB0421491C8AB20821104610
:101BA000FFF724F800BF4FF4804202EB0422521CDE
:101BB00091B20846FEF774FF0028F4D110BD10B5AD
:101BC0000446082201212046FFF768FC00BF0121DE
:101BD0002046FFF763FB0028F9D110BD0146CA0279
:101BE00002F5404290B270470146CA0202F5004237
:101BF00090B2704710B504464FF4804202EB0422C5
:101C0000263291B20846FEF797FF10BD10B5044684
:101C100026212046FFF780FB10BD10B504464FF487
:101C2000804202EB0422D21C91B20846FEF738FF34
:101C300010BD10B5044603212046FFF72FFB10BD51
:101C400010B504464FF4804202EB0422203291B2D8
:101C50000846FEF771FF10BD10B50446202120464E
:101C6000FFF75AFB10BD000070B5064602208A49F6
:101C70000871002088710220C87148714FF4E0504B
:101C800008608648FEF718FE06220A218348FEF700
:101C90005BFE06220B218148FEF756FE06220C2130
:101CA0007E48FEF751FE4FF440507B49086001200A
:101CB000087100208871022048717948FEF7FCFD08
:101CC0007848FFF79BF80020774908808880C88013
:101CD00008814FF400704881282088810020C88145
:101CE000072008824FF4827048806E48FFF7C0F8E2
:101CF00001216C48FFF776F814206C490870282001
:101D0000487050208870A120C8704220087185203A
:101D100048710A2088711420C87128200872502048
:101D20004872A12088724220C872852008730A2058
:101D300048734FF480515A48FEF729FE4FF4005182
:101D40005748FEF724FE57480C3000885849086071
:101D5000002054490C31088000BF524808300088E8
:101D600000F001000028F8D04E480C30008850499F
:101D700008604FF400514A48FEF70BFE002405E0CE
:101D80004848083000884A490860641CB4F5FA7F66
:101D9000F6DB4FF400514248FEF7F9FD4FF4805155
:101DA0003F48FEF7F6FD00252CE03E480C30008849
:101DB0003F4908603D48405D3A490C31088000BF0A
:101DC00038480830008800F001000028F8D0354875
:101DD0000C300088364908604FF400513048FEF757
:101DE000D8FD002405E02F480830008830490860FD
:101DF000641CB4F5FA7FF6DB4FF400512848FEF777
:101E0000C6FD6D1C0E2DD0DB4FF480512448FEF72B
:101E1000BEFD00212348FEF7E5FF2248FEF7EEFF56
:101E20000020214908804FF4006088800020C8808D
:101E300008814FF400704881282088810020C881E3
:101E4000072008824FF4827048801648FFF710F888
:101E500001211448FEF7C6FF4FF400511048FEF769
:101E600096FD10480C300088114908600D490C316E
:101E70000E8000BF0B480830008800F001000028E9
:101E8000F8D008480C300088094908604FF4005128
:101E90000348FEF77EFD70BD64000020000802408C
:101EA000000C0240003C00406802002043830020F8
:101EB00090000020FE48806840F48050FC49886013
:101EC0000121FC48FEF73EFF012141F21000FEF720
:101ED00069FF0121F848FEF745FF0120FEF72AFFC0
:101EE000F648006840F48070F44908600020F44926
:101EF00008710120C8717F200860F248FEF7DCFC01
:101F0000F14C282503E0641E0CB96D1EEE4CED4823
:101F1000006900F0100008B9002DF4DC35B900208C
:101F2000EA4988600120EA490880ACE00020E849DD
:101F30000880E6488068E749884257D101F09AFA5C
:101F40004FF48072D102E44801F0FAFA0020FFF762
:101F50008BFE00250020E149086001F08BFA002487
:101F60002DE0DA484FF480720169DB4801F0E8FAAD
:101F7000D648006900F58070D4490861D8482044EB
:101F8000D84908604FF48070FEF7ECFBD348006836
:101F900000F58070D1490860084600684CF2503165
:101FA00088420AD90020CD4908606D0045F001053E
:101FB0002846FFF759FE01F05DFA04F58074C34826
:101FC000C068A042CDD80020C04988604CF6CC4003
:101FD000C549086045F2555008600120486010204E
:101FE00088604AF6AA20086000BFFEE7B74880680C
:101FF000BE49884246D0BA480068BD490840B0F1A1
:10200000005F3FD1B648006AB4490860B448406AEE
:10201000B8490860B2483030B7490860AF48006836
:10202000B0F5503F00D92EE0B2480068D0B1012091
:10203000B249886000240AE0AF4800680068AF49F0
:102040000860AD480068001DAB490860641CA348E7
:1020500000688442F0D3A9480068A649096888420C
:1020600000D010E09E484068A54908600846006816
:10207000A44908609A49086880F3088800BFA1480D
:102080000068804700BF02208D49087100208871D8
:102090000220C87148714FF4E05008609A48FEF77A
:1020A0000BFC06220A219848FEF74EFC06220B2163
:1020B0009548FEF749FC06220C219348FEF744FCA4
:1020C0004FF440507E49086001200871002088715B
:1020D000022048718D48FEF7EFFB8D48FEF78EFE1B
:1020E00000208C4908808880C88008814FF40070E7
:1020F0004881282088810020C881072008824FF469
:10210000827048808248FEF7B3FE01218048FEF7C6
:1021100069FE14207049087028204870502088708B
:10212000A120C87042200871852048710A2088715A
:102130001420C8712820087250204872A12088728B
:102140004220C872852008730A2048734FF48051DA
:102150006E48FEF71CFC4FF400516C48FEF717FC6C
:102160006B480C3000886C490860002068490C31CD
:10217000088000BF66480830008800F00100002891
:10218000F8D063480C300088634908604FF4005170
:102190005E48FEF7FEFB002405E05D48083000883D
:1021A0005D490860641CB4F5FA7FF6DB4FF400511A
:1021B0005648FEF7ECFB4FF480515448FEF7E9FB1C
:1021C00000252CE052480C300088534908604248F2
:1021D000405D4F490C31088000BF4D4808300088F1
:1021E00000F001000028F8D049480C3000884A4926
:1021F00008604FF400514548FEF7CBFB002405E092
:1022000043480830008844490860641CB4F5FA7FEC
:10221000F6DB4FF400513D48FEF7B9FB6D1C0E2D67
:10222000D0DB4FF480513948FEF7B1FB002138482C
:10223000FEF7D8FD3648FEF7E1FD0020354908805D
:102240004FF4006088800020C88008814FF400703F
:102250004881282088810020C881072008824FF407
:10226000827048802A48FEF703FE01212848FEF7C5
:10227000B9FD0020124908710120C8717F20086053
:102280001048FEF719FB0F4801697F20884320F0B2
:102290001000224908600020214908601F4800788A
:1022A00000F0010000287DD01E481F4908603DE075
:1022B000002004E07F1064000180001000700040E6
:1022C000640000200010024040420F000040024025
:1022D0008E000020009125FC438300208000002018
:1022E00000000108E800002000300040715548124D
:1022F0000000FE2F840000208800002000300240F3
:10230000F4000020F000002000080240000C024011
:10231000003C00406802002090000020F8000020EF
:10232000FC000020BF1B000818000020F448F549FD
:102330000860F548F5490860F548F6490860F64830
:10234000F6490860F648F7490860F748F749086019
:10235000F748F8490860F848F8490860F848F9492A
:102360000860F948F9490860F948FA490860FA48EC
:10237000FA490860FA48FB490860FB48FB490860D5
:10238000FB48FC490860FC48FC490860FC48FD49E2
:102390000860FD48FD490860FD48006840F4804041
:1023A000FB4900E009E00860FFF7FAF8F848006828
:1023B00040F48050F649086040E0F648F64908606D
:1023C000F648D0490860F648D0490860F548D14938
:1023D0000860F548D1490860F448D2490860F448DB
:1023E000D2490860F348D3490860F348D3490860EC
:1023F000F248D4490860F248D4490860F148D54908
:102400000860F148D5490860F048D6490860F048AE
:10241000D6490860EF48D7490860EF48D7490860B7
:10242000EE48D8490860EE48D8490860D8480068A6
:1024300040F48050D6490860FFF7B2F8E9480088B8
:1024400010B1FEF7CFFD01E0FDF7C2FFE64880685E
:10245000E64988420CD1E448C06848B1E248C06807
:10246000E3490860E04840698860DF4800694860E7
:102470000020DD498860FEF7C1FADE490860DE48C9
:1024800000684008DD49B0FBF1F0401EDC490880DF
:1024900000204880401E48600020088188724FF06C
:1024A0008040FEF773FE01218807FEF763FEB848FF
:1024B000008800F4804010B1FFF766F901E0FFF7F3
:1024C00085F80121CF48FEF762FA00204FF08041E5
:1024D00048620846406ACC490844CC49086000BFBD
:1024E0004FF08040406AC94909688842F8D3012109
:1024F000C448FEF74EFA00204FF08041486208467B
:10250000406AC3490844C149086000BF4FF0804099
:10251000406ABE4909688842F8D30020BD49086076
:10252000B4480068B94908600846006842F2107172
:10253000B0FBF1F00404B5480068B0FBF1F201FB18
:102540001200B2490860084600684FF47A71B0FB87
:10255000F1F004EB0034AD480068B0FBF1F201FB90
:102560001200AA490860084600686421B0FBF1F037
:1025700004EB0024A5480068B0FBF1F201FB120057
:10258000A2490860084600680A21B0FBF1F004EB9C
:1025900000149E480068B0FBF1F201FB12009B4959
:1025A00008600846006820440860FA209A490870CC
:1025B000CE2048701020887094480068000CC870C5
:1025C00092480088000A08719048007848710846CF
:1025D0005C4909688847864868490968884784488B
:1025E00008305C49096888478148001D57490968D7
:1025F000884741F288305B490968884707205B4972
:10260000096888474D48006880474CF6CC408349AC
:10261000086045F255500860042048604FF47A7015
:1026200088604AF6AA20086000204FF08041486286
:102630000846406A7449084479490860002079498D
:102640000860F9E34AF6AA20744908604007406A26
:1026500073490968884251D900204FF0804148628F
:102660000846406A684908446D4908606D4800683A
:10267000401C6C4908600846006840F6B831884242
:102680000FD94CF6CC406549086045F255500860BA
:1026900001204860102088604AF6AA20086000BF28
:1026A000FEE761480068401C5F4908600846007802
:1026B00000F0040008B34FF400515C48FEF767F9DE
:1026C0005B4800885149086045F2555058490880D8
:1026D00000BF5748001F008800F001000028F8D014
:1026E00053480088494908604FF400514F48FEF7AD
:1026F00050F900204C490860C1E09BE0DEE000009A
:10270000193000081C0000208D3600082000002031
:102710008532000824000020651B000828000020E6
:10272000FB1900082C0000206B1900083000002065
:102730000D1C000834000020BB38000838000020C1
:10274000731A00083C000020733700084000002086
:102750005F38000844000020A73700084800002028
:10276000DF3700084C000020C3370008500000206D
:102770002F190008540000201338000858000020CA
:10278000591C00085C000020331C00086000002079
:10279000FC0000208D1B000818000020CF2F00082F
:1027A0004B360008293100081F1B00088919000852
:1027B00039190008F51B0008853800083D1A000883
:1027C0004D3700083938000899370008D13700081C
:1027D000B537000825190008ED370008411C00082E
:1027E0001B1C00088E00002000400240715548125A
:1027F000E4020020780000200000002040420F008A
:102800004002002000180240A08601009000002035
:1028100020A10700D8000020DC000020003000408C
:1028200094000020980000209C000020000C024032
:102830000C3C00404FF40051F748FEF7A8F8F74869
:102840000088F7490860F748008820B14AF6AA20B6
:10285000F249088002E00020F049088000BFEF48FC
:10286000001F008800F001000028F8D0EB48008825
:10287000EB4908604FF40051E748FEF78AF8E94851
:102880000088B0F57A7F19DDE6480088401EE549EA
:10289000088008460088B0F57A7F0FDC4CF6CC4003
:1028A000E149086045F25550086001204860102059
:1028B00088604AF6AA20086000BFFEE7DB4800688F
:1028C00000287DD0D9480068C01E062877D2DFE8EE
:1028D00000F0EAE976A5E803D5A1D848FEF742FB67
:1028E000F0B3FDF7D3FEF320FDF732FE02215820AE
:1028F000FDF734FEFDF79AFED149D248FFF7D4F830
:10290000D048FDF75DFCD04908600846008882B2D7
:10291000CC490720CD4B1B68984700204FF08041E1
:10292000486200BF4FF08040406A4CF2503188420C
:10293000F8D30720C6490968884700204FF0804136
:10294000486200BF4FF08040406A4CF250318842EC
:10295000F8D30020BF4988604CF6CC40B24900E073
:102960000CE0086045F255500860012048601020D6
:1029700088604AF6AA20086000BFFEE7B6A1AF480B
:10298000FEF7F0FAE8B1FDF781FEF320FDF7E0FD78
:1029900002214820FDF7E2FDFDF748FEA849A948BD
:1029A000FFF782F8A748FDF70BFCA7490860032052
:1029B0009E4908600020AB490860AB490860C6E149
:1029C000C6E1AAA19D48FEF7CDFAA8B1AA480068C1
:1029D000FDF780FE9A499B48FFF766F89948FDF796
:1029E000EFFB9949086003209049086000209D4949
:1029F00008609D490860AAE1A0484068A0490860B5
:102A00000020984908609D48C0689C494968401A60
:102A10008D49086003208549086098E18148008855
:102A2000F0BB98A18548FEF79DFA002871D0844933
:102A30008448FFF739F88348FDF7C2FB8A490860EC
:102A40000846008882B27F490720804B1B68984760
:102A500000204FF08041486200BF4FF08040406A44
:102A60004CF250318842F8D30720794909688847E9
:102A700000204FF08041486200BF4FF08040406A24
:102A80004CF250318842F8D30020724988604CF6ED
:102A9000CC406549086045F255500860012003E0CC
:102AA0000AE043E047E11BE14860102088604AF6F5
:102AB000AA20086000BFFEE760486F490860002454
:102AC0001BE06D4800680078212804D16A4800683E
:102AD000401C694908606848006800787D2800D17A
:102AE0000EE065480068FDF756FF564908556248F4
:102AF0000068801C60490860641CB4F5806FE0DBEE
:102B000000BF14B12046FDF72DFE4FF47F704549FC
:102B100008805F494B48FEF7C7FF4A48FDF750FB66
:102B20005149086004204149086010E13D4800888F
:102B3000B8BB58A14148FEF715FA98B34E48006853
:102B400000783A2803D0052038490860FFE04A4859
:102B50000068401C4849086032480088401C3149E0
:102B6000088045480068FDF716FF00064C490860DC
:102B700041480068801C4049086008460068FDF72D
:102B80000AFF4749096841EA0040454908603A4858
:102B90000068801C38490860414800684149086065
:102BA0000CE007E0FFE700202F49086005201F49DF
:102BB000086094E021483049086000BF002416E016
:102BC0002D48006800787D2804D02B4800680078E4
:102BD000212800D10EE028480068FDF7DCFE1949E5
:102BE000085525480068801C23490860641CB4F51A
:102BF000806FE5DB00BF14B12046FDF7B3FD1E4832
:102C00000068401C1C49086000202749086001201A
:102C10000649086000245FE0000C02400C3C0040C4
:102C2000900000208C00002000300040A800002010
:102C3000436C656172436F6E6600000044030020C0
:102C40006063000843830020B800002020000020BB
:102C50001800002000400240436C65617243616CC3
:102C600063000000B4000020AC00002053657450E5
:102C70003D7B313739360000EC000020C862000887
:102C8000CC00002072756E6D61696E3D7B000000A6
:102C9000B46300084669726D4845583D7B000000EA
:102CA000E4000020E8000020A40000209B48006809
:102CB000007828B19948006800789949085500E0E3
:102CC0000CE096480068401C9449086095480068EC
:102CD000401C94490860641CFA2CE7DB00BF36E016
:102CE00091480068B0F5FA7F24D99048006808BB85
:102CF000002414E08E4800688E49096888420CD28E
:102D00008D4800688A490968405C8C4908558848A4
:102D10000068401C8649086000E003E0641CB4F5CC
:102D2000967FE7DB00BF14B18048046002E0042016
:102D3000834908600BE07C480068B0F5006F05D15E
:102D40007A48006810B905207D49086000BF00BFBF
:102D500007207C490968884790B1132804D01728B8
:102D600029D01C280BD11AE0072077490968884729
:102D700000206C4908607549086071490860C9E025
:102D80000023502201210720714E3668B0470020F1
:102D9000644908606D49086069490860BAE0072025
:102DA0006C490968884700205E49086067490860E7
:102DB00063490860AEE007206749096888475A49B7
:102DC00008605F48006806287ED2DFE800F0030450
:102DD000A284859600BF072060490968884760493A
:102DE00008600846006840B308460068642801D9B6
:102DF000642008605A48008882B24948494B1B68E1
:102E0000C1180720574B1B6898474D48006840BBC6
:102E100043480078472811D14148407845280DD1D2
:102E20003F488078542809D13D48C078202805D1F2
:102E300008204349086018E06DE04BE0384800780E
:102E400050280FD1364840784F280BD1344880782D
:102E5000532807D13248C078542803D1012038497B
:102E6000086002E0052036490860354800680128FE
:102E700019D1002413E02B48006820442849085C3D
:102E8000212802D07D2808D103E007202C490860C2
:102E900003E006202A49086000BF00BF641C3048D8
:102EA00000688442E7D31F4800682D490968084438
:102EB0001C49086000201A491A4A126888541948A7
:102EC000006847F2FD7100E023E0884202D9052046
:102ED0001B4908601DE000BF1448006860B113483A
:102EE000008882B2154907201F4B1B6898470020B5
:102EF0000D4908600D4908600BE007201549096875
:102F00008847002007490860104908600C4908609C
:102F100000BF00BF00BFFFF795BB0000EC00002022
:102F200044030020A4000020C8000020AC000020C2
:102F3000B4000020B8000020CC0000204383002013
:102F4000A80000206000002030000020B000002019
:102F50002C000020180000205C000020340000201D
:102F6000800000201C000020200000202DE9F047F8
:102F70008246894616461C46C9F30A085046FEF7A3
:102F80002DFE00EB080508EB0400B0F5006F16DD20
:102F9000C8F500618FB2ABB23A463146184600F030
:102FA0008DFC3E44E11B8FB25046FEF717FE0546EE
:102FB0002B463A463146184600F080FC05E0ABB29D
:102FC00022463146184600F079FCBDE8F087F0B59E
:102FD00004460E4615460027002D1BDD2A463146C5
:102FE000204600F07FF84FF4804101EB0421491C9A
:102FF0008AB240211046FDF7F9FD00BF4FF4804230
:1030000002EB0422521C91B20846FDF749FD00284C
:10301000F4D12F463846F0BD2DE9F04381460F46E6
:1030200015462D490C6828214846FEF775F90646D5
:103030002A4800882A49096848833012207100BF55
:10304000207800F001000028FAD02079267100BF16
:10305000207800F001000028FAD020794FEA89009A
:10306000C01C002101EBC000207100BF207800F0DF
:1030700001000028FAD020794FF000080EE000206F
:10308000207100BF207800F001000028FAD02079DC
:1030900038707F1C08F101001FFA80F8A845EEDBAC
:1030A0000E4909880E4A1268118371198EB2324690
:1030B00028214846FEF72EFA402201214846FEF715
:1030C000EDF900BF01214846FEF7E8F80028F9D1E4
:1030D0002846BDE8F0830000B4010020B8010020BC
:1030E000B0010020F0B504460E4615464FF480426C
:1030F00002EB0422283291B20846FDF71DFD074677
:103100002B46324639462046FFF730FF79198FB2F9
:103110004FF4804101EB042128318AB23946104630
:10312000FDF7AEFDF0BD00002DE9FC4304468946E5
:10313000154698464FF4804202EB0422283291B2A1
:103140000846FDF7F9FC07464FF4804202EB0422E3
:1031500091B20846FDF7A4FC00F00700022804D055
:1031600003282BD0042856D144E008236A46394668
:103170002046FFF7FBFE07F1080087B29DF800002C
:1031800028709DF8010068709DF80200A8709DF8F5
:103190000300E8709DF80400A8F800009DF8050001
:1031A00098F8001000EB0120A8F800009DF80660D8
:1031B0009DF8070000EB062086B22DE006236A4644
:1031C00039462046FFF7D2FEB81D87B29DF80000B1
:1031D00028709DF8010068709DF80200A8709DF8A5
:1031E0000300E8709DF804609DF8050000EB0620E0
:1031F00086B211E002236A4639462046FFF7B6FE42
:10320000B81C87B29DF800609DF8010000EB062015
:10321000801E86B200E000BF00BFB6F5007F06DA70
:1032200033464A4639462046FFF7A0FE00E0002616
:10323000B9198FB212490F804FF4804101EB04217C
:1032400028318AB239461046FDF71AFD4FF4804105
:1032500001EB0421491C8AB240211046FDF7C6FC4F
:1032600000BF4FF4804202EB0422521C91B2084688
:10327000FDF716FC0028F4D13046BDE8FC830000C1
:10328000AC0100202DE9FF4B814615469846764952
:103290000C6828214846FEF73FF807467348008827
:1032A0007349096848833812207100BF207800F004
:1032B00001000028FAD02079277100BF207800F0A3
:1032C00001000028FAD020794FEA8900C01C0021B3
:1032D00001EBC000207100BF207800F00100002841
:1032E000FAD020790020207100BF207800F0010082
:1032F0000028FAD0207928700020207100BF2078A3
:1033000000F001000028FAD020796D1C2870002000
:10331000207100BF207800F001000028FAD0207949
:103320006D1C28700020207100BF207800F0010083
:103330000028FAD020796D1C28700020207100BF71
:10334000207800F001000028FAD02079A8F80000C9
:103350000020207100BF207800F001000028FAD082
:10336000207998F8001000EB0120A8F80000002058
:10337000207100BF207800F001000028FAD02079E9
:1033800006460020207100BF207800F001000028D0
:10339000FAD0207900EB062086B234480088344900
:1033A0000968088307F1080087B2B6F5007F40DCA2
:1033B0002E4800882E49096848833812207100BFC2
:1033C000207800F001000028FAD02079277100BF92
:1033D000207800F001000028FAD020794FEA890017
:1033E000C01C002101EBC000207100BF207800F05C
:1033F00001000028FAD020794FF0000B12E00020E5
:10340000207100BF207800F001000028FAD0207958
:103410002179019801700198401C01900BF1010085
:103420001FFA80FBB345EADB1048008810490968A1
:103430000883B9198FB23A4628214846FEF76AF840
:10344000402201214846FEF729F800BF01214846E5
:10345000FDF724FF0028F9D1B6F5007F02DD04B0A6
:10346000BDE8F08B3046FAE7B4010020B801002037
:10347000B001002010B502202C490871002088718D
:103480000220C87148714FF4E05008602848FDF7E9
:1034900013FA06220A212648FDF756FA06220B21C6
:1034A0002348FDF751FA06220C212148FDF74CFA7A
:1034B0004BF210001D49086001200871002088713E
:1034C000022048711B48FDF7F7F910211948FDF754
:1034D0005EFA4FF400411748FDF75BFA4FF40041E4
:1034E0001448FDF756FA00211348FDF77BFC1248FB
:1034F000FDF784FC00201149088088800220C880E4
:103500000120088140024881082088810020C8816C
:10351000072008824FF4827048800748FDF7A8FC16
:1035200001210548FDF75EFC10BD0000640000208D
:1035300000080240000C0240003C004068020020ED
:1035400070B505460C46164600F042F84FF40041AF
:103550001048FDF71CFA032000F01EF8C4F30740E2
:1035600000F01AF8C4F3072000F016F8E0B200F0FB
:1035700013F804E0A52000F00FF828706D1C30004F
:10358000A6F101018EB2F5D14FF400410148FDF7DB
:1035900000FA70BD000C024010B5044600BF0221C5
:1035A0000A48FDF757FC0028F9D021460748FDF7E7
:1035B0005DFC00BF01210548FDF74CFC0028F9D057
:1035C0000248FDF750FCC0B210BD0000003C0040B6
:1035D00010B500244FF400410A48FDF7D8F9052042
:1035E000FFF7DAFF00BFA520FFF7D6FF044604F07F
:1035F00001000028F7D14FF400410248FDF7C9F956
:1036000010BD0000000C0240F0B504460F46154600
:103610004FF4804202EB0422243291B20846FDF7B7
:103620008BFA06462B4632463946204600F0FAF918
:1036300071198EB24FF4804101EB042124318AB21A
:1036400031461046FDF71CFBF0BD70B504460D4633
:103650001646324629462046FFF7D6FF4FF48041F2
:1036600001EB0421491C8AB220211046FDF7BEFA65
:1036700000BF4FF4804202EB0422521C91B2084674
:10368000FDF70EFA0028F4D170BD00002DE9F043DB
:103690008046894617462A490C6824214046FDF792
:1036A0003BFE0546274800882749096848832812B9
:1036B000207100BF207800F001000028FAD02079A6
:1036C000257100BF207800F001000028FAD0207991
:1036D0004FEA8800801C042101EBC000207100BF6C
:1036E000207800F001000028FAD0207900260AE0B6
:1036F00019F80600207100BF207800F001000028B2
:10370000FAD02079761CBE42F2DB0E4909880E4AB7
:1037100012681183E9198DB22A4624214046FDF72B
:10372000F9FE202201214046FDF7B8FE00BF01212D
:103730004046FDF7B3FD0028F9D1BDE8F083000055
:10374000B4010020B8010020B001002010B50446EB
:1037500021780120FDF74AFA61780220FDF746FA48
:10376000A1780320FDF742FAE1780420FDF73EFA44
:1037700010BD10B5044621780120FDF715FE6178D3
:103780000220FDF711FEA1780320FDF70DFEE17880
:103790000420FDF709FE10BD10B5044621460020A7
:1037A000FDF724FA10BD10B5044621460020FDF7B0
:1037B000FBFD10BD10B5044621461920FDF716FA91
:1037C00010BD10B5044621461B20FDF7EDFD10BDD0
:1037D00010B5044621461720FDF752FA10BD10B56A
:1037E000044621461920FDF717FE10BD10B504460A
:1037F00021780F20FDF7FAF961781020FDF7F6F92E
:10380000A1781120FDF7F2F9E1781220FDF7EEF929
:1038100010BD10B5044621780F20FDF7C5FD617875
:103820001020FDF7C1FDA1781120FDF7BDFDE17865
:103830001220FDF7B9FD10BD10B504462178052012
:10384000FDF7D4F961780620FDF7D0F9A1780720BB
:10385000FDF7CCF9E1780820FDF7C8F910BD10B5E7
:10386000044621780520FDF79FFD61780620FDF7CD
:103870009BFDA1780720FDF797FDE1780820FDF773
:1038800093FD10BD10B5002414E04FF4804101EB0E
:1038900004211F318AB202211046FDF7A7F94FF427
:1038A000804101EB04211E318AB202211046FDF74E
:1038B0009DF9641C082CE8DB10BD704770B5034609
:1038C0000C4600214FF48040264D28805818000AED
:1038D000254D287300BF2448007A00F0010000281D
:1038E000F9D02148007B58181F4D287300BF1E488F
:1038F000007A00F001000028F9D01B48007BC2F3D9
:103900000620194D287300BF1748007A00F0010007
:103910000028F9D01448007B134D2A7300BF1248C9
:10392000007A00F001000028F9D00F48007B002148
:103930000EE000200C4D287300BF0B48007A00F009
:1039400001000028F9D0084D287B6054481C81B242
:103950009142EEDB4FF48045024EB61E3580104694
:1039600070BD00001A0C02400030014070B50346E3
:103970000C4600210AB9002070BD4FF48040274D4D
:1039800028805818000A264D287300BF2448007A62
:1039900000F001000028F9D02148007B5818204D84
:1039A000287300BF1E48007A00F001000028F9D0FB
:1039B0001B48007BC2F3062040F08000184D28739E
:1039C00000BF1748007A00F001000028F9D0144821
:1039D000007B134D2A7300BF1148007A00F00100EC
:1039E0000028F9D00E48007B00210DE0605C0C4DF2
:1039F000287300BF0A48007A00F001000028F9D0BF
:103A00000748007B481C81B29142EFDB4FF48045B0
:103A1000024EB61E35801046AEE700001A0C02407A
:103A2000003001402DE9F0478246884691461C4609
:103A3000C9F30A075046FEF7D7F8C5193819B0F58B
:103A4000006F16DDC7F500618EB2ABB2324641465B
:103A50001846FFF78BFFB044A11B8EB25046FEF70D
:103A6000C3F805462B46324641461846FFF77EFF0F
:103A700005E0ABB2224641461846FFF777FFBDE8A6
:103A8000F087000053494E44303A30392E30372EFB
:103A9000323031382020393A313500485454502FD3
:103AA000312E3120323030204F4B0D0A5365727663
:103AB00065723A2053696E636F6D440D0A436F6EF1
:103AC00074656E742D547970653A20746578742F1E
:103AD00068746D6C3B20636861727365743D555406
:103AE000462D380D0A436F6E6E656374696F6E3ACA
:103AF000204B6565702D416C6976650D0A436163E5
:103B000068652D436F6E74726F6C3A206E6F2D7303
:103B1000746F72652C206E6F2D63616368652C2055
:103B20006D7573742D726576616C69646174650D71
:103B30000A457870697265733A204D6F6E2C203299
:103B400036204A756C20313939372030353A3030DB
:103B50003A303020474D540D0A0D0A3C21444F4362
:103B6000545950452068746D6C3E3C68746D6C3ED1
:103B70003C686561643E3C6D657461206368617298
:103B80007365743D5554462D383E3C7469746C65BC
:103B90003ED09ED0B1D0BDD0BED0B2D0BBD0B5D07B
:103BA000BDD0B8D0B520D0BFD180D0BED0B3D180E9
:103BB000D0B0D0BCD0BCD18B20D0BAD0BED0BDD17B
:103BC00082D180D0BED0BBD0BBD0B5D180D0B03CEC
:103BD0002F7469746C653E3C7374796C65207479DC
:103BE00070653D746578742F6373733E2A7B6D61D5
:103BF0007267696E3A303B70616464696E673A302F
:103C00003B626F782D73697A696E673A626F72648E
:103C100065722D626F787D626F64797B666F6E74FA
:103C20002D73697A653A2E3735656D3B666F6E7414
:103C30002D66616D696C793A417269616C2C4865D9
:103C40006C7665746963612C73616E732D73657234
:103C500069663B636F6C6F723A233333333B6D613C
:103C60007267696E3A31656D7D6469767B6D6172EC
:103C700067696E3A31656D20303B6C696E652D6801
:103C800065696768743A313530257D68317B6D61CF
:103C90007267696E3A3020302031656D3B666F6E19
:103CA000742D73697A653A323030257D68312C681D
:103CB000327B666F6E742D7765696768743A34304D
:103CC000307D68327B6D617267696E3A32656D2056
:103CD000302031656D3B666F6E742D73697A653A7D
:103CE000313530257D696E7075747B6D61726769E1
:103CF0006E3A302032656D3B70616464696E673A7C
:103D000035707820313270783B626F726465723A38
:103D100031707820736F6C696420236262623B6645
:103D20006F6E743A696E68657269743B6C696E6532
:103D30002D6865696768743A6E6F726D616C3B637C
:103D40006F6C6F723A233434347D696E7075743AD7
:103D5000666F6375737B626F726465722D636F6CDF
:103D60006F723A233032383864317D627574746F03
:103D70006E7B70616464696E673A367078203132A8
:103D800070783B6261636B67726F756E643A233063
:103D900032383864313B636F6C6F723A2366666603
:103DA0003B626F726465723A6E6F6E653B666F6EF2
:103DB000743A696E68657269743B6C696E652D68EA
:103DC00065696768743A6E6F726D616C3B6F75748C
:103DD0006C696E653A6E6F6E657D627574746F6E38
:103DE0003A686F7665727B6261636B67726F756E3E
:103DF000642D636F6C6F723A233032393865613BE2
:103E0000626F782D736861646F773A302031707813
:103E100020337078207267626128302C302C302C6F
:103E20002E3132292C302031707820327078207277
:103E300067626128302C302C302C2E3234293B63C1
:103E40007572736F723A706F696E7465727D6275A8
:103E500074746F6E3A6163746976657B6261636BDB
:103E600067726F756E642D636F6C6F723A233032B8
:103E7000373862383B626F782D736861646F773AC8
:103E800030202D317078203370782072676261287D
:103E9000302C302C302C2E3132292C30202D31700A
:103EA0007820327078207267626128302C302C3094
:103EB0002C2E3234297D627574746F6E3A3A2D6DF2
:103EC0006F7A2D666F6375732D696E6E65727B6296
:103ED0006F726465723A307D617B636F6C6F723AAA
:103EE000233232323B746578742D6465636F72617E
:103EF00074696F6E3A6E6F6E657D23666163746F71
:103F000072792D646174617B646973706C61793A54
:103F10006E6F6E657D23666163746F72792D646167
:103F20007461206C6162656C7B646973706C61792B
:103F30003A696E6C696E652D626C6F636B3B776975
:103F40006474683A383070787D23666163746F7288
:103F5000792D6461746120696E7075747B77696412
:103F600074683A33303070783B6D617267696E3ACD
:103F7000302031656D203020307D23666163746FA1
:103F800072792D737472696E67732D6C6973747BAB
:103F9000706F736974696F6E3A6162736F6C757478
:103FA000653B6C6566743A34363570783B746F7077
:103FB0003A32343070783B70616464696E673A31CC
:103FC0003070783B6261636B67726F756E642D63EE
:103FD0006F6C6F723A236565657D23666163746FEC
:103FE00072792D737472696E67732D6C69737420A6
:103FF0006C697B6C6973742D7374796C652D74793D
:1040000070653A6E6F6E653B70616464696E673AA5
:1040100035707820303B626F726465722D626F7408
:10402000746F6D3A31707820736F6C69642023620D
:1040300062623B637572736F723A706F696E74651A
:10404000727D237374617475737B636F6C6F723AE6
:104050007265643B666F6E742D73697A653A3135AB
:1040600030253B746578742D616C69676E3A6365C1
:104070006E7465727D23696E7374616C6C7B766996
:10408000736962696C6974793A68696464656E7DA4
:104090003C2F7374796C653E3C2F686561643E3CCF
:1040A000626F64793E3C68313ED0A0D0B5D0B6D0C6
:1040B000B8D0BC20D0BED0B1D0BDD0BED0B2D0BB65
:1040C000D0B5D0BDD0B8D18F20D0BFD180D0BED098
:1040D000B3D180D0B0D0BCD0BCD18B20D0BAD0BEB0
:1040E000D0BDD182D180D0BED0BBD0BBD0B5D18025
:1040F0003C6120687265663D6A61766173637269CE
:1041000070743A766F69642830293B2069643D6693
:104110006163746F72792D646174612D73686F7758
:104120003ED0B03C2F613E3C2F68313E3C64697606
:104130003E3C627574746F6E20747970653D627573
:1041400074746F6E2069643D657869742074697455
:104150006C653D22D092D18BD0B9D182D0B820D01D
:10416000B8D0B720D180D0B5D0B6D0B8D0BCD0B000
:1041700020D0BFD180D0BED0B3D180D0B0D0BCD001
:10418000BCD0B8D180D0BED0B2D0B0D0BDD0B8D124
:104190008F223ED092D18BD0B9D182D0B820D0B866
:1041A000D0B720D180D0B5D0B6D0B8D0BCD0B02058
:1041B000D0BED0B1D0BDD0BED0B2D0BBD0B5D0BDB6
:1041C000D0B8D18F20D0BFD180D0BED0B3D180D0D5
:1041D000B0D0BCD0BCD18B3C2F627574746F6E3E76
:1041E0003C2F6469763E3C6469762069643D666173
:1041F00063746F72792D646174613E3C68323ED0A5
:10420000A3D181D182D0B0D0BDD0BED0B2D0BAD0EF
:10421000B020D0B7D0B0D0B2D0BED0B4D181D0BA57
:10422000D0B8D18520D0B4D0B0D0BDD0BDD18BD145
:10423000853C2F68323E3C6469763E3C6C61626529
:104240006C20666F723D666163746F72792D646174
:1042500074612D70773ED09FD0B0D180D0BED0BBDE
:10426000D18C3A3C2F6C6162656C3E3C696E707516
:104270007420747970653D746578742069643D6656
:104280006163746F72792D646174612D70773E3C47
:104290002F6469763E3C6469763E3C6C6162656C75
:1042A00020666F723D666163746F72792D6461740C
:1042B000612D7365723ED0A1D0B5D1802FD0BD3AAB
:1042C0003C2F6C6162656C3E3C696E707574207445
:1042D0007970653D746578742069643D66616374C6
:1042E0006F72792D646174612D7365723E3C6275E5
:1042F00074746F6E20747970653D627574746F6E3E
:104300002069643D666163746F72792D64617461C4
:104310002D7365722D696E633E2B3C2F627574742C
:104320006F6E3E3C2F6469763E3C6469763E3C6C21
:104330006162656C20666F723D666163746F72794D
:104340002D646174612D7374723ED0A1D182D180CD
:10435000D0BED0BAD0B03A3C2F6C6162656C3E3CA6
:10436000696E70757420747970653D746578742019
:1043700069643D666163746F72792D646174612D47
:104380007374723E3C627574746F6E2074797065DC
:104390003D627574746F6E2069643D666163746F0D
:1043A00072792D646174612D7374722D6C697374EC
:1043B0003E266C743B2D2D2D3C2F627574746F6EF0
:1043C0003E3C2F6469763E3C6469763E3C6C61629B
:1043D000656C20666F723D666163746F72792D64DF
:1043E0006174612D73656E643E3C2F6C6162656C17
:1043F0003E3C627574746F6E20747970653D6275B1
:1044000074746F6E2069643D666163746F72792D98
:10441000646174612D73656E643ED0A3D181D182D5
:10442000D0B0D0BDD0BED0B2D0B8D182D18C3C2FCC
:10443000627574746F6E3E3C2F6469763E3C2F64E7
:1044400069763E3C68323ED092D0BED181D181D1D6
:1044500082D0B0D0BDD0BED0B2D0BBD0B5D0BDD050
:10446000B8D0B520D0BAD0BED0BDD182D180D0BE18
:10447000D0BBD0BBD0B5D180D0B03C2F68323E3C51
:104480006469763E3C627574746F6E2074797065F1
:104490003D627574746F6E2069643D636C65617212
:1044A0002D63616C63207469746C653D22D0A3D068
:1044B000B4D0B0D0BBD0B8D182D18C20D0BFD18005
:1044C000D0BED0B3D180D0B0D0BCD0BCD18320D0AE
:1044D000B4D0BED180D0B0D181D187D0B5D182D077
:1044E000B0223ED0A3D0B4D0B0D0BBD0B8D182D10E
:1044F0008C20D0BFD180D0BED0B3D180D0B0D0BCC2
:10450000D0BCD18320D0B4D0BED180D0B0D181D1A5
:1045100087D0B5D182D0B03C2F627574746F6E3E77
:10452000203C627574746F6E20747970653D62759D
:1045300074746F6E2069643D636C6561722D636F86
:104540006E666967207469746C653D22D0A3D0B42F
:10455000D0B0D0BBD0B8D182D18C20D0BAD0BED010
:10456000BDD184D0B8D0B3D183D180D0B0D186D0E2
:10457000B8D18E223ED0A3D0B4D0B0D0BBD0B8D169
:1045800082D18C20D0BAD0BED0BDD184D0B8D0B327
:10459000D183D180D0B0D186D0B8D18E3C2F627576
:1045A00074746F6E3E3C2F6469763E3C68323ED038
:1045B0009ED0B1D0BDD0BED0B2D0BBD0B5D0BDD0D2
:1045C000B8D0B520D184D0B0D0B9D0BBD0B020D035
:1045D000BFD180D0BED0B3D180D0B0D0BCD0BCD100
:1045E0008B3C2F68323E3C6469763ED092D18BD0B2
:1045F000B1D0B5D180D0B8D182D0B520D184D0B0DF
:10460000D0B9D0BB20D0BFD180D0BED0B3D180D064
:10461000B0D0BCD0BCD18B3A3C696E70757420743C
:104620007970653D66696C652069643D66696C6595
:10463000206175746F636F6D706C6574653D6F6636
:10464000663E3C2F6469763E3C6469762069643D31
:1046500066696C652D696E666F3E3C2F6469763EB7
:104660003C6469763E3C627574746F6E2074797038
:10467000653D627574746F6E2069643D696E737414
:10468000616C6C207469746C653D22D0A3D181D1BA
:1046900082D0B0D0BDD0BED0B2D0B8D182D18C2023
:1046A000D0B2D18BD0B1D180D0B0D0BDD0BDD1836C
:1046B000D18E20D0BFD180D0BED0B3D180D0B0D0E9
:1046C000BCD0BCD183223ED0A3D181D182D0B0D086
:1046D000BDD0BED0B2D0B8D182D18C20D0B2D18BD7
:1046E000D0B1D180D0B0D0BDD0BDD183D18E20D0BB
:1046F000BFD180D0BED0B3D180D0B0D0BCD0BCD1DF
:10470000833C2F627574746F6E3E3C2F6469763EF5
:104710003C6469762069643D7374617475733E3CD2
:104720002F6469763E3C736372697074207479708B
:10473000653D746578742F6A617661736372697020
:10474000743E2166756E6374696F6E2874297B668A
:10475000756E6374696F6E206E2872297B69662896
:10476000655B725D2972657475726E20655B725D42
:104770002E6578706F7274733B76617220693D6547
:104780005B725D3D7B693A722C6C3A21312C657805
:10479000706F7274733A7B7D7D3B72657475726E57
:1047A00020745B725D2E63616C6C28692E65787075
:1047B0006F7274732C692C692E6578706F727473C4
:1047C0002C6E292C692E6C3D21302C692E65787059
:1047D0006F7274737D76617220653D7B7D3B6E2EBA
:1047E0006D3D742C6E2E633D652C6E2E643D66759A
:1047F0006E6374696F6E28742C652C72297B6E2E23
:104800006F28742C65297C7C4F626A6563742E6402
:104810006566696E6550726F706572747928742C64
:10482000652C7B636F6E666967757261626C653A51
:1048300021312C656E756D657261626C653A21304F
:104840002C6765743A727D297D2C6E2E6E3D6675DF
:104850006E6374696F6E2874297B76617220653D82
:10486000742626742E5F5F65734D6F64756C653FAB
:1048700066756E6374696F6E28297B7265747572D4
:104880006E20745B2264656661756C74225D7D3A8E
:1048900066756E6374696F6E28297B7265747572B4
:1048A0006E20747D3B72657475726E206E2E642866
:1048B000652C2261222C65292C657D2C6E2E6F3D86
:1048C00066756E6374696F6E28742C6E297B7265D1
:1048D0007475726E204F626A6563742E70726F74A5
:1048E0006F747970652E6861734F776E50726F7058
:1048F000657274792E63616C6C28742C6E297D2C22
:104900006E2E703D222F222C6E286E2E733D302984
:104910007D285B66756E6374696F6E28742C6E2CCF
:1049200065297B66756E6374696F6E2072287429C1
:104930007B69662832213D3D742E6C656E67746814
:104940002972657475726E206E756C6C3B7661723F
:10495000206E3D7061727365496E7428742C313617
:10496000293B72657475726E2069734E614E286EB4
:10497000293F6E756C6C3A6E7D66756E6374696FF7
:104980006E206928297B666F722876617220743DDB
:104990005B66756E6374696F6E28297B72657475CA
:1049A000726E206E657720584D4C48747470526555
:1049B00071756573747D2C66756E6374696F6E288E
:1049C000297B72657475726E206E65772041637401
:1049D000697665584F626A65637428224D73786DF5
:1049E0006C322E584D4C4854545022297D2C6675FB
:1049F0006E6374696F6E28297B72657475726E20A0
:104A00006E657720416374697665584F626A6563A5
:104A10007428224D73786D6C332E584D4C48545485
:104A20005022297D2C66756E6374696F6E28297B10
:104A300072657475726E206E657720416374697655
:104A400065584F626A65637428224D6963726F739B
:104A50006F66742E584D4C4854545022297D5D2C5D
:104A60006E3D21312C653D303B653C742E6C656E8E
:104A70006774683B652B2B297B7472797B6E3D7460
:104A80005B655D28297D63617463682872297B6397
:104A90006F6E74696E75657D627265616B7D72653E
:104AA0007475726E206E7D66756E6374696F6E20AC
:104AB0006F2874297B72657475726E20646F6375DC
:104AC0006D656E742E676574456C656D656E7442B8
:104AD0007949642874297D66756E6374696F6E20E8
:104AE000612874297B666F7228766172206E2C654E
:104AF0003D742E73706C697428223A303230303035
:104B000030303422292C723D5B5D2C693D313B6E87
:104B10003D655B692B2B5D3B297B766172206F3D88
:104B20006E2E737562737472696E6728302C342927
:104B30002C613D7061727365496E74286F2C313041
:104B4000293B6966282128613C3830307C7C613EF5
:104B500039303029297B76617220633D6E2E737067
:104B60006C697428225C6E22293B722E6C656E671C
:104B700074687C7C722E7075736828223A222B6FC1
:104B8000293B666F7228766172206C2C753D323B32
:104B90006C3D635B752B2B5D3B297B7661722073CB
:104BA0003D6C2E736C69636528392C2D33293B725B
:104BB0002E707573682873292C3726757C7C722EAD
:104BC0007075736828222122297D7D7D4E3D722ECD
:104BD0006A6F696E282222292C5A3D4E2E73706C02
:104BE000697428222122292E6A6F696E28222229BF
:104BF0007D66756E6374696F6E206328742C6E29F0
:104C00007B76617220653D742B322A6E2C693D657E
:104C10002B312C6F3D72285A2E63686172417428C3
:104C200065292B5A2E636861724174286929293BD2
:104C300072657475726E20537472696E672E667237
:104C40006F6D43686172436F6465286F297D667577
:104C50006E6374696F6E206C28742C6E297B6E2BCA
:104C60003D31323B76617220653D7B747970653AE7
:104C7000742C643A7061727365496E742863286E8F
:104C80002C30292B63286E2C31292C3130292C6DA6
:104C90003A7061727365496E742863286E2C3329EB
:104CA0002B63286E2C34292C3130292C793A7061F1
:104CB000727365496E742863286E2C36292B63281D
:104CC0006E2C37292B63286E2C38292B63286E2CE9
:104CD00039292C3130292C683A7061727365496E1C
:104CE000742863286E2C3131292B63286E2C3132C5
:104CF000292C3130292C693A7061727365496E74C0
:104D00002863286E2C3134292B63286E2C313529E9
:104D10002C3130297D3B72657475726E20652E745E
:104D20007970652B223A222B652E642E6C656164A6
:104D3000696E675A65726F28292B222E222B652EE9
:104D40006D2E6C656164696E675A65726F28292BD8
:104D5000222E222B652E792E6C656164696E675A4E
:104D600065726F28292B2220222B652E682E6C65F8
:104D70006164696E675A65726F28292B223A222B6B
:104D8000652E692E6C656164696E675A65726F285D
:104D9000297D66756E6374696F6E20752874297B32
:104DA0006F282266696C652D696E666F22292E69EF
:104DB0006E6E657248544D4C3D747D66756E6374BD
:104DC000696F6E20732874297B6F28227374617455
:104DD000757322292E696E6E657248544D4C3D7470
:104DE0002E7265706C616365282F5C6E2F67692C6D
:104DF000223C6272202F3E22297D66756E637469A3
:104E00006F6E206628297B76617220743D6F2822A0
:104E100066696C6522292E66696C65735B305D3B43
:104E200069662821742972657475726E20766F69BF
:104E3000642075282222293B766172206E3D27D09E
:104E400092D18BD0B1D180D0B0D0BD20D184D0B0A0
:104E5000D0B9D0BB203C656D3E22272B742E6E61ED
:104E60006D652B27223C2F656D3E2C20272B287447
:104E70002E73697A652F31303234292E746F46696A
:104E800078656428292B2220D0BAD0B12E222C6537
:104E90003D6E65772046696C655265616465723B5D
:104EA000652E726561644173546578742874292C89
:104EB000652E6F6E6C6F61643D66756E6374696FAD
:104EC0006E2874297B6128742E7461726765742E54
:104ED000726573756C74293B76617220653D5A2E3C
:104EE000696E6465784F662848292C723D5A2E6990
:104EF0006E6465784F662858293B696628653C30A2
:104F00007C7C723C302972657475726E2075286ED7
:104F10002B223C6272202F3E3C7374726F6E673E90
:104F2000D09DD0B5D0BAD0BED180D180D0B5D0BAC6
:104F3000D182D0BDD18BD0B920D184D0B0D0B9D05E
:104F4000BB20D0BFD180D0BED0B3D180D0B0D0BC38
:104F5000D0BCD18B213C2F7374726F6E673E2229B7
:104F60002C766F6964286F2822696E7374616C6C8B
:104F700022292E7374796C652E7669736962696C67
:104F80006974793D2268696464656E22293B7661A3
:104F90007220693D6C284F2C65292C633D6C286A72
:104FA0002C72293B75286E2B223C6272202F3ED03A
:104FB0009AD0BED180D180D0B5D0BAD182D0BDD167
:104FC0008BD0B920D184D0B0D0B9D0BB20D0BFD144
:104FD00080D0BED0B3D180D0B0D0BCD0BCD18B21DA
:104FE0003C6272202F3E3C6272202F3ED092D0B5A0
:104FF000D180D181D0B8D18F20D0BFD180D0BED0C8
:10500000B3D180D0B0D0BCD0BCD18B20D0BAD0BE70
:10501000D0BDD182D180D0BED0BBD0BBD0B5D180E5
:10502000D0B03A203C7374726F6E673E222B692BAE
:10503000223C2F7374726F6E673E2C3C6272202F7D
:105040003ED092D0B5D180D181D0B8D18F20D0BF01
:10505000D180D0BED0B3D180D0B0D0BCD0BCD18BA9
:1050600020D0BAD0BED0BDD184D0B8D0B3D183D1F6
:1050700080D0B0D182D0BED180D0B03A203C737401
:10508000726F6E673E222B632B223C2F7374726FFC
:105090006E673E2E22292C6F2822696E7374616C14
:1050A0006C22292E7374796C652E76697369626936
:1050B0006C6974793D2276697369626C65227D7DC5
:1050C00066756E6374696F6E206428742C6E297B1C
:1050D00076617220653D6928293B652E6F6E726589
:1050E00061647973746174656368616E67653D6658
:1050F000756E6374696F6E28297B343D3D3D652E66
:1051000072656164795374617465262628636C65E1
:10511000617254696D656F75742872292C6E26262C
:105120006E2829297D2C652E6F70656E2822706F80
:105130007374222C222F222C2130292C652E73658A
:10514000745265717565737448656164657228226F
:10515000436F6E74656E742D54797065222C2261D4
:1051600070706C69636174696F6E2F782D777777D3
:105170002D666F726D2D75726C656E636F646564FC
:1051800022292C652E73656E642874292C732822BD
:10519000D092D18BD0BFD0BED0BBD0BDD18FD0B537
:1051A000D182D181D18F20D0BED0BFD0B5D180D017
:1051B000B0D186D0B8D18F2C20D0BFD0BED0B6D041
:1051C000B0D0BBD183D0B9D181D182D0B02C20D086
:1051D000B6D0B4D0B8D182D0B52E2E2E22293B76AF
:1051E000617220723D73657454696D656F757428C2
:1051F00066756E6374696F6E28297B652E61626FB8
:10520000727428292C732822D09AD0BED0BDD182A6
:10521000D180D0BED0BBD0BBD0B5D18020D0BDD046
:10522000B520D0BED182D0B2D0B5D187D0B0D0B564
:10523000D18222297D2C336534297D66756E637495
:10524000696F6E207628742C6E297B7661722065DA
:105250003D6928293B652E6F6E72656164797374B0
:105260006174656368616E67653D66756E637469D8
:105270006F6E28297B343D3D3D652E7265616479F2
:105280005374617465262628636C65617254696D78
:10529000656F75742872292C6E26266E2829297D43
:1052A0002C652E6F70656E2822676574222C222F64
:1052B0003F222B742C2130292C652E73656E6428B7
:1052C000292C732822D092D18BD0BFD0BED0BBD096
:1052D000BDD18FD0B5D182D181D18F20D0BED0BFEA
:1052E000D0B5D180D0B0D186D0B8D18F2C20D0BF4E
:1052F000D0BED0B6D0B0D0BBD183D0B9D181D1820D
:10530000D0B02C20D0B6D0B4D0B8D182D0B52E2E0B
:105310002E22293B76617220723D73657454696D4B
:10532000656F75742866756E6374696F6E28297B66
:10533000652E61626F727428292C732822D09AD04E
:10534000BED0BDD182D180D0BED0BBD0BBD0B5D174
:105350008020D0BDD0B520D0BED182D0B2D0B5D1C2
:1053600087D0B0D0B5D18222297D2C316534297DFA
:1053700066756E6374696F6E207028297B732822AE
:10538000D09ED0BFD0B5D180D0B0D186D0B8D18F8B
:1053900020D0B2D18BD0BFD0BED0BBD0BDD0B5D085
:1053A000BDD0B05C6ED094D0B0D0BDD0BDD0B0D1A7
:1053B0008F20D181D182D180D0B0D0BDD0B8D1865C
:1053C000D0B020D0BED0B1D0BDD0BED0B2D0B8D138
:1053D00082D181D18F20D187D0B5D180D0B5D0B73F
:1053E000203520D181D0B5D0BAD183D0BDD0B42260
:1053F000292C73657454696D656F75742866756EB4
:105400006374696F6E28297B77696E646F772E6C81
:105410006F636174696F6E2E72656C6F61642829A9
:105420007D2C356533297D66756E6374696F6E20DA
:105430007928297B732822D09ED0BFD0B5D180D0C7
:10544000B0D186D0B8D18F20D0B2D18BD0BFD0BE52
:10545000D0BBD0BDD0B5D0BDD0B05C6ED09FD0B5E4
:10546000D180D0B5D0BDD0B0D0BFD180D0B0D0B277
:10547000D0BBD0B5D0BDD0B8D0B520D0BDD0B02035
:10548000D0B1D0B0D0B7D0BED0B2D18BD0B920D0AF
:10549000B0D0B4D180D0B5D18120D0BAD0BED0BDEB
:1054A000D182D180D0BED0BBD0BBD0B5D180D0B05E
:1054B0002028222B502B222920D187D0B5D180D073
:1054C000B5D0B7203520D181D0B5D0BAD183D0BDE9
:1054D000D0B422292C73657454696D656F75742876
:1054E00066756E6374696F6E28297B77696E646F69
:1054F000772E6C6F636174696F6E3D22687474708F
:105500003A2F2F222B502B222F227D2C3565332929
:105510007D66756E6374696F6E206728297B7328BA
:1055200022D09ED0BFD0B5D180D0B0D186D0B8D156
:105530008F20D0B2D18BD0BFD0BED0BBD0BDD0B524
:10554000D0BDD0B022297D66756E6374696F6E2000
:105550006D28297B696628216F282266696C65227F
:10556000292E66696C65735B305D7C7C214E2972E7
:10557000657475726E20766F696420732822D0A3DB
:10558000D0BAD0B0D0B6D0B8D182D0B520D0BAD0B1
:10559000BED180D180D0B5D0BAD182D0BDD18BD090
:1055A000B920D184D0B0D0B9D0BB20D0BFD180D069
:1055B000BED0B3D180D0B0D0BCD0BCD18B22293BDF
:1055C00064284D2B227B222B4E2B227D222C7029EE
:1055D0007D66756E6374696F6E206828297B636FC2
:1055E0006E6669726D2822D09FD0BED0B4D182D0B1
:1055F000B2D0B5D180D0B4D0B8D182D0B520D0B29D
:10560000D18BD185D0BED0B420D0B8D0B720D18036
:10561000D0B5D0B6D0B8D0BCD0B020D0BED0B1D0EC
:10562000BDD0BED0B2D0BBD0B5D0BDD0B8D18F2008
:10563000D0BFD180D0BED0B3D180D0B0D0BCD0BC90
:10564000D18B20D0BAD0BED0BDD182D180D0BED037
:10565000BBD0BBD0B5D180D0B022293F6428462C26
:1056600070293A616C6572742822D09ED0BFD0B583
:10567000D180D0B0D186D0B8D18F20D0BED182D049
:10568000BCD0B5D0BDD0B5D0BDD0B022297D667517
:105690006E6374696F6E206228297B766172207454
:1056A0003D70726F6D70742827D092D0BDD0B8D085
:1056B000BCD0B0D0BDD0B8D0B52120D09FD180D043
:1056C000BED0B3D180D0B0D0BCD0BCD0B020D0B48C
:1056D000D0BED180D0B0D181D187D0B5D182D0B069
:1056E00020D0B1D183D0B4D0B5D18220D183D0B471
:1056F000D0B0D0BBD0B5D0BDD0B020D0B1D0B5D017
:10570000B720D0B2D0BED0B7D0BCD0BED0B6D0BDFE
:10571000D0BED181D182D0B820D0B2D0BED181D17B
:1057200081D182D0B0D0BDD0BED0B2D0BBD0B5D0A8
:10573000BDD0B8D18F5C6ED094D0BBD18F20D0BFFC
:10574000D0BED182D0B2D0B5D180D0B6D0B4D0B591
:10575000D0BDD0B8D18F20D0B2D0B2D0B5D0B4D0D7
:10576000B8D182D0B520D0B220D0BFD0BED0BBD06F
:10577000B520D181D0BBD0BED0B2D0BE2022D0A324
:10578000D094D090D09BD098D0A2D0AC22272C22FD
:1057900022293B74262622D183D0B4D0B0D0BBD0EE
:1057A000B8D182D18C223D3D3D742E746F4C6F7701
:1057B00065724361736528293F76286B2C67293A07
:1057C000616C6572742822D09ED0BFD0B5D180D0D4
:1057D000B0D186D0B8D18F20D0BED182D0BCD0B5C8
:1057E000D0BDD0B5D0BDD0B022297D66756E6374B2
:1057F000696F6E207728297B76617220743D707204
:105800006F6D70742822D092D0BDD0B8D0BCD0B00B
:10581000D0BDD0B8D0B52120D09AD0BED0BDD184D3
:10582000D0B8D0B3D183D180D0B0D186D0B8D18F09
:1058300020D0BAD0BED0BDD182D180D0BED0BBD016
:10584000BBD0B5D180D0B020D0B1D183D0B4D0B549
:10585000D18220D183D0B4D0B0D0BBD0B5D0BDD010
:10586000B020D0B1D0B5D0B720D0B2D0BED0B7D054
:10587000BCD0BED0B6D0BDD0BED181D182D0B820F0
:10588000D0B2D0BED181D181D182D0B0D0BDD0BE76
:10589000D0B2D0BBD0B5D0BDD0B8D18F5C6E49509E
:1058A0002DD0B0D0B4D180D0B5D18120D0BAD0BE67
:1058B000D0BDD182D180D0BED0BBD0BBD0B5D1803D
:1058C000D0B020D0B1D183D0B4D0B5D18220D18393
:1058D000D181D182D0B0D0BDD0BED0B2D0BBD0B5F6
:1058E000D0BD20D0BFD0BE20D183D0BCD0BED0BBD5
:1058F000D187D0B0D0BDD0B8D18E202D20222B5052
:105900002B275C6ED094D0BBD18F20D0BFD0BED11E
:1059100082D0B2D0B5D180D0B6D0B4D0B5D0BDD0C1
:10592000B8D18F20D0B2D0B2D0B5D0B4D0B8D18257
:10593000D0B520D0B220D0BFD0BED0BBD0B520D102
:1059400081D0BBD0BED0B2D0BE2022D0A3D094D0C4
:1059500090D09BD098D0A2D0AC22272C2222293BD9
:1059600074262622D183D0B4D0B0D0BBD0B8D18297
:10597000D18C223D3D3D742E746F4C6F7765724320
:1059800061736528293F76284C2C79293A616C652A
:1059900072742822D09ED0BFD0B5D180D0B0D1862D
:1059A000D0B8D18F20D0BED182D0BCD0B5D0BDD0A0
:1059B000B5D0BDD0B022297D66756E6374696F6EF7
:1059C000205428297B6F2822666163746F72792DB9
:1059D0006461746122292E7374796C652E64697315
:1059E000706C61793D22626C6F636B227D66756EAF
:1059F0006374696F6E204328297B76617220743D41
:105A00006F2822666163746F72792D646174612DF1
:105A1000707722292E76616C75652C6E3D6F282279
:105A2000666163746F72792D646174612D73657240
:105A300022292E76616C75652C653D6F2822666182
:105A400063746F72792D646174612D73747222298D
:105A50002E76616C75653B69662821747C7C216EAD
:105A60007C7C21652972657475726E20766F69641D
:105A700020616C6572742822D094D0BED0BBD0B6A1
:105A8000D0BDD18B20D0B1D18BD182D18C20D0B7D9
:105A9000D0B0D0BFD0BED0BBD0BDD0B5D0BDD18BE3
:105AA00020D0B2D181D0B520D0BFD0BED0BBD18F55
:105AB0002C20D0BED0BFD0B5D180D0B0D186D0B848
:105AC000D18F20D0BED182D0BCD0B5D0BDD0B5D082
:105AD000BDD0B022293B666F72283B6E2E6C656E7E
:105AE0006774683C363B296E3D2230222B6E3B6347
:105AF0006F6E6669726D2822D09FD0BED0B4D182FD
:105B0000D0B2D0B5D180D0B4D0B8D182D0B520D168
:105B100083D181D182D0B0D0BDD0BED0B2D0BAD1E5
:105B20008320D0B7D0B0D0B2D0BED0B4D181D0BA5B
:105B3000D0B8D18520D0B4D0B0D0BDD0BDD18BD11C
:105B40008522293F7628412B227B222B742B223A57
:105B500053222B6E2B652B227D222C67293A616CF8
:105B60006572742822D09ED0BFD0B5D180D0B0D17C
:105B700086D0B8D18F20D0BED182D0BCD0B5D0BD18
:105B8000D0B5D0BDD0B022297D66756E6374696FC3
:105B90006E207828297B76617220743D6F282266FA
:105BA0006163746F72792D646174612D7365722203
:105BB000293B742E76616C75653D70617273654921
:105BC0006E7428742E76616C75652C3130292B31FA
:105BD0002C742E666F63757328297D66756E6374E9
:105BE000696F6E204528297B76617220742C6E2C9B
:105BF000653D646F63756D656E742E637265617467
:105C000065456C656D656E742822756C22293B664E
:105C10006F7228652E69643D22666163746F7279C4
:105C20002D737472696E67732D6C697374222C7492
:105C30003D303B6E3D535B742B2B5D3B29652E69DC
:105C40006E6E657248544D4C2B3D273C6C69206943
:105C5000643D22666163746F72792D737472696E2C
:105C600067732D6C6973742D272B742B2722206486
:105C70006174612D737472696E673D22272B6E5BB0
:105C8000315D2B27223E272B6E5B305D2B223C2F74
:105C90006C693E223B666F7228646F63756D656E3A
:105CA000742E626F64792E617070656E64436869EA
:105CB0006C642865292C743D303B6E3D535B742B1E
:105CC0002B5D3B2952286F2822666163746F7279BD
:105CD0002D737472696E67732D6C6973742D222B2A
:105CE00074292C22636C69636B222C49297D6675AB
:105CF0006E6374696F6E204928297B766172207407
:105D00003D746869732E6765744174747269627555
:105D100074652822646174612D737472696E6722E0
:105D2000293B646F63756D656E742E626F64792EA6
:105D300072656D6F76654368696C64286F282266AA
:105D40006163746F72792D737472696E67732D6CF1
:105D50006973742229293B766172206E3D6F282277
:105D6000666163746F72792D646174612D737472EE
:105D700022293B6E2E76616C75653D742C6E2E6605
:105D80006F63757328297D652831293B7661722000
:105D90004D3D224669726D4845583D222C463D22B4
:105DA00072756E6D61696E3D7B317D222C4C3D229A
:105DB000436C656172436F6E66222C6B3D22436CAF
:105DC00065617243616C63222C413D2253657450BE
:105DD0003D222C483D223533343934453434333078
:105DE0003341222C4F3D2253494E30222C583D2224
:105DF000353334393445343435373341222C6A3D18
:105E00002253494E57222C503D223139322E313601
:105E1000382E312E32222C533D5B5B22D0A1D0B8DC
:105E2000D0BDD0BAD0BED0BC2DD09432222C222CE2
:105E300044322C45322C43342C463031303430340B
:105E4000303235225D2C5B22D0A1D0B8D0BDD0BA83
:105E5000D0BED0BC2DD09433222C222C44332C45E0
:105E6000322C43342C463031303430343032352209
:105E70005D2C5B22D0A1D0B8D0BDD0BAD0BED0BCF2
:105E80002DD094D09A32222C222C4B322C45322CFD
:105E900043342C46303130343034303235225D2CAE
:105EA0005B22D0A1D0B8D0BDD0BAD0BED0BC2DD04E
:105EB00094D09AD09F222C222C4D322C45312C4349
:105EC000342C547331322C547530322C46303130EE
:105ED000343034303235225D2C5B22D0A1D0B8D0A2
:105EE000BDD0BAD0BED0BC2DD0942F3355222C2299
:105EF0002C55322C45312C43322C46303130343045
:105F000034303235225D5D2C5A3D222C222C4E3D00
:105F100022223B4E756D6265722E70726F746F74C3
:105F20007970652E6C656164696E675A65726F3D44
:105F300066756E6374696F6E28297B7265747572FD
:105F40006E20746869733C31303F2230222B7468B4
:105F500069733A22222B746869737D3B76617220E3
:105F6000523D66756E6374696F6E28742C6E2C6575
:105F7000297B742E6164644576656E744C69737414
:105F8000656E65723F742E6164644576656E744C0F
:105F9000697374656E6572286E2C652C2131293AFF
:105FA000742E6174746163684576656E743F742EF7
:105FB0006174746163684576656E7428226F6E2221
:105FC0002B6E2C65293A745B226F6E222B6E5D3D21
:105FD000657D3B77696E646F772E46696C65262612
:105FE00077696E646F772E46696C6552656164658A
:105FF00072262677696E646F772E46696C654C69E8
:1060000073747C7C28732822D092D0B0D18820D0A1
:10601000B1D180D0B0D183D0B7D0B5D18020D0BDA0
:10602000D0B520D0BFD0BED0B4D0B4D0B5D180D000
:10603000B6D0B8D0B2D0B0D0B5D18220D0BCD0B517
:10604000D185D0B0D0BDD0B8D0B7D0BC20D0BFD0D3
:10605000B5D180D0B5D0BFD180D0BED0B3D180D0A3
:10606000B0D0BCD0BCD0B8D180D0BED0B2D0B0D02F
:10607000BDD0B8D18F20D0BAD0BED0BDD182D18012
:10608000D0BED0BBD0BBD0B5D180D0B02E5C6E5CC2
:106090006ED092D0BED181D0BFD0BED0BBD18CD07B
:1060A000B7D183D0B9D182D0B5D181D18C20D0BE27
:1060B000D0B4D0BDD0B8D0BC20D0B8D0B720D1811A
:1060C000D0BBD0B5D0B4D183D18ED189D0B8D18551
:1060D00020D0B1D180D0B0D183D0B7D0B5D180D0CD
:1060E000BED0B23A5C6E496E7465726E65742045BE
:1060F00078706C6F7265722031312E3020D0B820EC
:10610000D0B2D18BD188D0B52C5C6E4D6F7A696CD2
:106110006C612046697265666F7820332E3620D018
:10612000B820D0B2D18BD188D0B52C5C6E476F6FC0
:10613000676C65204368726F6D6520372E3020D004
:10614000B820D0B2D18BD188D0B52C5C6E4F7065A1
:1061500072612031312E353020D0B820D0B2D18BB1
:10616000D188D0B52E22292C6F282266696C652231
:10617000292E64697361626C65643D2130292C525B
:10618000286F282266696C6522292C226368616E5B
:106190006765222C66292C52286F28226661637459
:1061A0006F72792D646174612D73686F7722292C69
:1061B00022636C69636B222C54292C52286F28228D
:1061C000666163746F72792D646174612D73657299
:1061D0002D696E6322292C22636C69636B222C78F3
:1061E000292C52286F2822666163746F72792D649E
:1061F0006174612D7374722D6C69737422292C2261
:10620000636C69636B222C45292C52286F28226607
:106210006163746F72792D646174612D73656E644E
:1062200022292C22636C69636B222C43292C52286F
:106230006F2822696E7374616C6C22292C22636C46
:1062400069636B222C6D292C52286F2822636C65A0
:1062500061722D63616C6322292C22636C69636B0C
:10626000222C62292C52286F2822636C6561722DC2
:10627000636F6E66696722292C22636C69636B22E7
:106280002C77292C52286F28226578697422292CB2
:1062900022636C69636B222C68297D2C66756E63A2
:1062A00074696F6E28742C6E297B7D5D293B3C2FB1
:1062B0007363726970743E3C2F626F64793E3C2F49
:1062C00068746D6C3E0000008699CE2E9B3A0008E3
:1062D00000000000C56200080040404040404040CF
:1062E00040404141414141404040404040404040A9
:1062F000404040404040404040050202020202024D
:10630000020202020202020202202020202020209B
:1063100020202002020202020202909090909090AF
:10632000101010101010101010101010101010106D
:1063300010101010020202020202888888888888E1
:1063400008080808080808080808080808080808CD
:10635000080808080202020240000000D962000892
:10636000485454502F312E3120323030204F4B20A2
:106370000D0A436F6E6E656374696F6E3A20636CCD
:106380006F73650D0A4163636573732D436F6E749C
:10639000726F6C2D416C6C6F772D4F726967696EEF
:1063A0003A2A0D0A0D0A205265616479210D0A0D01
:1063B0000A000000485454502F312E312032303022
:1063C000204F4B200D0A436F6E6E656374696F6ECC
:1063D0003A20636C6F73650D0A4163636573732DB7
:1063E000436F6E74726F6C2D416C6C6F772D4F72B2
:1063F0006967696E3A2A0D0A0D0A00001C640008DC
:1064000000000020400200003E030008B8640008BD
:1064100040020020308E0000E41A000811847A0344
:106420000A0009ED010203040607080912351201EA
:106430001B4003052A41052A42052A43052A440533
:106440002A45052A46052A470513402082089A4115
:106450000C9A420C9A430C9A440C9A450C9A460C9E
:106460009A470C111209022C02232E011B03090466
:106470001A29041A49041A69041A89041AA9041A5F
:10648000C90422E933200A2A26052B202A0A2905D5
:106490002B204A0A29052B206A0A29052B208A0A63
:1064A00029052B20AA0A29052B20CA0A29052B20F9
:0864B000EA0A2905CA09A2004D
:040000050800018965
:00000001FF
